:1000000025009F0C0200080C0600000C2600660666
:10001000070A6607090A880988098809880988097A
:100020008809880988096607460B880988098109B3
:10003000810981096607900A81096607940A810986
:100040006607A10A81096607AC0A81096607B70A33
:1000500081096607C20A81096607CD0A8109660718
:10006000D80A81096607E30A81096607EE0A810951
:100070006607F90A81096607040B810966070F0BF9
:10008000810966071A0B81096607250B8109660736
:10009000300B810966073B0B81096607460B810916
:1000A00066074A0B81096607550B81096607600BD5
:1000B000810966076B0B81096607760B8109660764
:1000C000810B810966078C0B81096607970B8109F3
:1000D0006607A20B81096607AD0B81096607B80B9D
:1000E00081096607C30B81096607CE0B8109660784
:1000F000D90B81096607E40B81096607EF0B8109BB
:10010000FC0B050C2700E702830A860A00000008A2
:10011000170C29000000E9028A0A8E0A0000000874
:10012000A3050009A304070A180C3700A30500095A
:100130007D09A304F702960AA30539090609A30459
:10014000070A170C3700A30500097D0906090909EC
:10015000A304F702A30A070A170C3700A305000936
:10016000720906091009A304F702AE0A070A170C60
:100170003700A3050009680906091809A304F70256
:10018000B90A070A170C3700A30500095F09060919
:100190002109A304F702C40A070A170C3700A305B4
:1001A0000009540906092609A304F702CF0A070A21
:1001B000170C3700A30500094A0906092C09A304F6
:1001C000F702DA0A070A170C3700A30500094109EC
:1001D00006092609A304F702E50A070A170C3700E7
:1001E000A3050009390906093909A304F702F00A31
:1001F000070A170C3700A30500093209060941094F
:10020000A304F702FB0A070A170C3700A30500092D
:100210002C0906094A09A304F702060B070A170C62
:100220003700A3050009260906095409A304F702AB
:10023000110B070A170C3700A3050009210906094D
:100240005F09A304F7021C0B070A170C3700A3056C
:100250000009180906095409A304F702270B070A25
:10026000170C3700A3050009100906097209A30439
:10027000F702320B070A170C3700A305000909091A
:1002800006097D09A304F7023D0B070AA305060929
:10029000A304070A170C3700A30503090909060977
:1002A0007D09A304F7024C0B070A170C3700A305BE
:1002B0000309100906097209A304F702570B070A7C
:1002C000170C3700A3050309180906096809A304D8
:1002D000F702620B070A170C3700A305030921096F
:1002E00006095F09A304F7026D0B070A170C370014
:1002F000A3050309260906095409A304F702780B8C
:10030000070A170C3700A30503092C0906094A0937
:10031000A304F702830B070A170C3700A305030990
:10032000320906094109A304F7028E0B070A170CCC
:100330003700A3050309390906093909A304F7029F
:10034000990B070A170C3700A30503094109060991
:100350003209A304F702A40B070A170C3700A30500
:1003600003094A0906092C09A304F702AF0B070A7F
:10037000170C3700A3050309540906092609A3042D
:10038000F702BA0B070A170C3700A30503095F0928
:1003900006092109A304F702C50B070A170C370049
:1003A000A3050309680906091809A304F702D00B7D
:1003B000070A170C3700A30503097209060910097B
:1003C000A304F702DB0B070A170C3700A305030988
:1003D0007D0906090909A304F702E60B070A180CB0
:1003E0003700A30503097D09A304F702F10BA30558
:1003F00039090609A304070AA3050309A304070A88
:10040000030C26000008300C26000008000C260013
:1004100000080B0C28000000E8020B0A000000088E
:10042000170C29000000E902120A160A0000000851
:10043000230C2A000000EA021A0A1E0A1F0A000002
:100440000008410C2B00EB02230A0008510C2C0081
:10045000EC02280A2B0A0008620C2D00ED022E0A7D
:1004600000000008720C2E00EE02340A370A000069
:100470000008820C2F00EF023B0A3E0A3F0A0000F0
:100480000008920C3000F002430A460A470A480A64
:1004900000000008A20C3100F1024C0A4F0A500A79
:1004A000510A520A00000008B20C3200F202560A49
:1004B000590A5A0A5B0A5C0A5D0A00000008C40C6B
:1004C0003300F302610A640A650A660A0000000844
:1004D000D40C3400F4026A0A6D0A6E0A6F0A700ABC
:1004E00000000008E40C3500F502740A770A780A67
:1004F000790A7A0A7B0A00000008F40C3600F6023A
:100500007F0A820A830A840A850A860A870A00000B
:020510000008E1
:0207FE00640C89
:021FFE00EA0FE8
:00000001FF
